:020000020000FC
:060000000C942900189584
:02000800189549
:06000C000C947802189527
:0200140018953D
:02001800189539
:02001C00189535
:02002000189531
:0200240018952D
:02002800189529
:02002C00189525
:02003000189521
:0200340018951D
:060038000C945F01189515
:02004000189511
:0200440018950D
:100048000C94A7020C94C5011895F8940FE50DBF00
:1000580004E00EBF01E00093850000E000938600F5
:1000680001E00093880001E0009387000AE0009314
:10007800830000E00093940000270093890081E04A
:1000880090E00E94170A0093820082E090E00E94AC
:10009800170A00938400009182000F3F11F40E9418
:1000A800040A00E00BBB00E00ABB00E008BB08EF55
:1000B80007BB00E005BB0FEF04BB00E002BB0FEF7E
:1000C80001BB0E94100B00E00093800000E0006C70
:1000D80007B90FE806B9369A00E002BF05E003BF8A
:1000E80009B7026009BF00E004BD01E005BD09B71A
:1000F800006809BF04B70F7B04BF0BB700620BBFD2
:10010800789401E00093850000E000938600C3988E
:10011800C4980E94C1020E94C60A04E60E94F3091C
:100128000E942F0820916E0030916F003695279518
:1001380036952795243568F3209170003091710029
:100148003695279536952795243518F32091720012
:100158003091730036952795369527952435C8F242
:10016800209174003091750036952795369527951E
:10017800243578F2209176003091770036952795CE
:1001880036952795283628F202E00093850000E08E
:1001980000938600C39AC4980E94C1020E94C60AAE
:1001A80004E60E94F3090E942F082091680030910C
:1001B800690036952795369527952E3468F303E020
:1001C8000093850000E000938600C39AC49A0E94B9
:1001D800C1020E94C60A04E60E94F3090E942F0881
:1001E80020916A0030916B003695279536952795B2
:1001F800213668F320916C0030916D003695279573
:1002080036952795283818F304E00093850001E017
:10021800009386000E94C1020E94C60A04E60E945A
:10022800F3090E94720906B300FF0E9452080E9457
:100238002F0808B304FB26F403FB16F40C940E01F4
:10024800C398C4980E94C1020E94C60A04E60E948C
:10025800F3090E942F0820916800309169003695B3
:100268002795369527952C306CF720916A003091A8
:100278006B0036952795369527952C301CF72091DD
:100288006C0030916D0036952795369527952C3062
:10029800CCF606E00093850000E000938600C39842
:1002A800C4980E94C1020E94C60A04E60E94F3098B
:1002B8000E942F08F6CF0F930FB70F931F932F931A
:1002C8003F934F93AF93BF9304B115B120917E0034
:1002D80030917F00200F311F20937E0030937F00E4
:1002E800409180004395409380004130D1F14134E2
:1002F800E9F520917E0030917F0036952795369557
:1003080027953695279536952795369527953695C9
:100318002795A0E6B0E007B10770073099F4AEE67C
:10032800B0E0009181000770102F1395177010939B
:100338008100110F110F110F110F110F48B34871E0
:10034800412B48BB10E0000FA00FB11F2D933D9328
:1003580000E00093800007B103950770006C07B9AF
:1003680005C000E000937E0000937F00369ABF919D
:10037800AF914F913F912F911F910F910FBF0F9107
:1003880018950F930FB70F931F932F933F934F9386
:1003980000918A00039500938A000431C9F400276C
:1003A80000938A00009186000130D1F00BEE009393
:1003B8008C0000938D0000938E0000938F0000E066
:1003C8000093900000939100009392000093930093
:1003D8004F913F912F911F910F910FBF0F9118953A
:1003E8003091820010916000209161002695179548
:1003F8002695179500918C00432F46951695411B1D
:1004080069F04595459509F44395041B1AE025EFD5
:10041800011708F40AE0201708F405EF00938C0090
:1004280040939000109162002091630026951795E3
:100438002695179500918D00432F46951695411BDB
:1004480069F04595459509F44395041B1AE025EF95
:10045800011708F40AE0201708F405EF00938D004F
:10046800409391001091640020916500269517959E
:100478002695179500918E00432F46951695411B9A
:1004880069F04595459509F44395041B1AE025EF55
:10049800011708F40AE0201708F405EF00938E000E
:1004A8004093920010916600209167002695179559
:1004B8002695179500918F00432F46951695411B59
:1004C80069F04595459509F44395041B1AE025EF15
:1004D800011708F40AE0201708F405EF00938F00CD
:1004E800409393000C94EC010F930FB70F931F9355
:1004F80000918B00039500938B00003009F49098CD
:1005080010918C00011709F4909A003009F4919821
:1005180010918D00011709F4919A0058003009F4E0
:10052800929810918E00011709F4929A003009F4FC
:10053800939810918F00011709F4939A1F910F91C6
:100548000FBF0F9118950F930FB70F931F9310912B
:10055800890006B30670023021F0043011F01A95B4
:1005680001C013951093890010E404B7012704BF54
:100578001F910F910FBF0F9118950F931F932F93F2
:10058800AF93BF93CF93DF93EF93FF9310919400B2
:1005980006B300FD11271395153111F40C942900A9
:1005A800109394000091850010E0000F111FECEEED
:1005B800FBE0E00FF11F05911591E02FF12FC5E940
:1005C800D0E00E942C03009188000A9510E0000FEB
:1005D800111F000F111FEEEAFDE0E00FF11F05915A
:1005E8001591E02FF12FC0EBD0E000E209950091C2
:1005F800880010E0000F111F000F111FEEEAFDE048
:10060800E00FF11F05911591E02FF12FCBECD0E011
:100618000FE7099500918800039510E0000F111F5E
:10062800000F111FEEEAFDE0E00FF11F0591159193
:10063800E02FF12FC6EED0E000E20995FF91EF918F
:10064800DF91CF91BF91AF912F911F910F91089595
:100658000F931F93CF93DF93EF93FF931BE10591C4
:1006680009931A95E1F7FF91EF91DF91CF911F91CF
:100678000F910895E2E1FEE00E942C032396009179
:1006880068001091690043E060E0E2E8F5E10E944B
:10069800770A289600916C0010916D0043E060E0A5
:1006A800E2E8F5E10E94770A299600916A00109124
:1006B8006B0043E060E0E2E8F5E10E94770A089504
:1006C800EEE2FEE00E942C0321960091600010915A
:1006D800610044E061E0EEE6F5E10E94770A2696C3
:1006E80000918C0010E043E060E0E4E6F5E10E9450
:1006F800770A08E20883259600916200109163004A
:1007080044E061E0EEE6F5E10E94770A2696009162
:100718008D0010E043E060E0E4E6F5E10E94770A2E
:1007280008E208830895EAE4FEE00E942C0321967B
:10073800009164001091650044E061E0EEE6F5E1A7
:100748000E94770A269600918E0010E043E060E050
:10075800E4E6F5E10E94770A08E20883259600910D
:1007680066001091670044E061E0EEE6F5E10E9462
:10077800770A269600918F0010E043E060E0E4E6F7
:10078800F5E10E94770A08E208830895E6E6FEE0AC
:100798000E942C03229600916E0010916F0044E095
:1007A80061E0E8E7F5E10E94770A0DE20883269602
:1007B80000918C0010E043E060E0E4E6F5E10E947F
:1007C800770A08E20883269600917000109171005C
:1007D80044E061E0E8E7F5E10E94770A0DE208836A
:1007E800269600918D0010E043E060E0E4E6F5E134
:1007F8000E94770A08E208830895E2E8FEE00E9472
:100808002C032296009172001091730044E061E07D
:10081800E8E7F5E10E94770A0DE208832696009141
:100828008E0010E043E060E0E4E6F5E10E94770A1C
:1008380008E208832696009174001091750044E040
:1008480061E0E8E7F5E10E94770A0DE20883269661
:1008580000918F0010E043E060E0E4E6F5E10E94DB
:10086800770A08E208830895EEE9FEE00E942C0367
:100878002196009160001091610044E061E0EEE68D
:10088800F5E10E94770A269600916E0010916F009C
:1008980044E061E0E8E7F5E10E94770A0DE20883A9
:1008A8002596009162001091630044E061E0EEE655
:1008B800F5E10E94770A2696009170001091710068
:1008C80044E061E0E8E7F5E10E94770A0DE2088379
:1008D8000895EAEBFEE00E942C0321960091640043
:1008E8001091650044E061E0EEE6F5E10E94770AC8
:1008F8002696009172001091730044E061E0E8E7E9
:10090800F5E10E94770A0DE20883259600916600BA
:100918001091670044E061E0EEE6F5E10E94770A95
:100928002696009174001091750044E061E0E8E7B4
:10093800F5E10E94770A0DE208830895E6EDFEE0EE
:100948000E942C03239600918C0010E043E060E0A5
:10095800E4E6F5E10E94770A239600918D0010E005
:1009680043E060E0E4E6F5E10E94770A239600910F
:100978008E0010E043E060E0E4E6F5E10E94770ACB
:10098800239600918F0010E043E060E0E4E6F5E193
:100998000E94770A2896009176001091770044E02B
:1009A80061E0E8E7F5E10E94770A0DE2088308951F
:1009B800E2EFFEE00E942C03DE015A960C932D967E
:1009C8000091820010E0000F111F000F111F44E07A
:1009D80061E0EEE6F5E10E94770A0895EEE0FFE0B7
:1009E8000E942C03DE015A960C932D9600918400E8
:1009F80010E0000F111F000F111F44E061E0EEE648
:100A0800F5E10E94770A0895EAE2FFE00E942C03CC
:100A18006A9608830895E6E4FFE00E942C036A962C
:100A280008830895E2E6FFE00E942C036A96088393
:100A38000895EEE7FFE00E942C036A960883089564
:100A4800EAE9FFE00E942C03DE015A960C932E96E9
:100A580000918700002321F00FE41EE420E203C088
:100A68000FE416E426E40993199329930895E6EB15
:100A7800FFE00E942C0326962091610000916000FF
:100A88000E94540A269620916300009162000E94F9
:100A9800540A269620916500009164000E94540A29
:100AA800269620916700009166000E94540A0895D6
:100AB800E2EDFFE00E942C03269620916900009148
:100AC80068000E94540A269620916B0000916A00E3
:100AD8000E94540A269620916D0000916C000E9495
:100AE800540A26960DE4099305E5099308E5099348
:100AF8000895EEEEFFE00E942C03269620916F00E9
:100B080000916E000E94540A26962091710000916F
:100B180070000E94540A269620917300009172007A
:100B28000E94540A269620917500009174000E9434
:100B3800540A0895EAE0F0E10E942C0326962091D9
:100B48007700009176000E94540A26962091790039
:100B5800009178000E94540A269620917B0000910B
:100B68007A000E94540A269620917D0000917C000C
:100B78000E94540A0895E6E2F0E10E942C032796A9
:100B880000918C000E94390A269600918D000E94DF
:100B9800390A269600918E000E94390A26960091FD
:100BA8008F000E94390A0895E2E4F0E10E942C03C4
:100BB8002796009190000E94390A2696009191008C
:100BC8000E94390A2696009192000E94390A2696B8
:100BD800009193000E94390A0895E6EFFDE00E9413
:100BE8002C0308950A0C260C420C5E0C7A0C960C09
:100BF800B20CCE0CEA0C060D220D3E0D5A0D760DE8
:100C0800920D20202020202020202020202020207D
:100C18002020202020202020202020202000576174
:100C28006974696E6720666F722067726964312023
:100C3800737570706C792E2E2E0057616974696E09
:100C48006720666F7220707265616D7020706F77B3
:100C580065722E2E2E005374617274696E6720754A
:100C6800702E2E2E20202020202020202020202002
:100C7800200052756E6E696E672E2E2E2020202061
:100C88002020202020202020202020202000536801
:100C9800757474696E6720646F776E2E2E2E20200F
:100CA80020202020202020202000506C65617365C2
:100CB80020737769746368206F66662E2E2E202055
:100CC8002020202020004661696C7572652049202B
:100CD8004B6174686F6465203136323520233120CA
:100CE80020004661696C7572652049204B61746803
:100CF8006F6465203136323520233220200046616A
:100D0800696C7572652049204B6174686F64652051
:100D1800313632352023332020004661696C7572E4
:100D2800652049204B6174686F646520313632351F
:100D38002023342020004661696C75726520552097
:100D4800477269643120737570706C792020202097
:100D580020004661696C7572652055205072656186
:100D68006D7020737570706C7920202020004661AA
:100D7800696C7572652055204772696432207375F5
:100D880070706C792020202020004661696C757293
:100D980065205520506C61746520737570706C798E
:100DA8002020202020003E037F0838047F086D049F
:100DB8007F08A2047F08DC048008F204B70808054D
:100DC800EC080F05EE081605F3081D053B09240578
:100DD8004909F1057F083B057F085C057F087D050B
:100DE8007F089E057F08BF057F08D8057F0820205B
:100DF80020202020202020202020202020202020EB
:100E08002020202020202020200055763D5F5F5F95
:100E18002C2055613D5F5F5F2C205567323D5F5F39
:100E28005F20202056004C205F5F2C5F20285F5FEA
:100E38002529205F5F2C5F20285F5F252920206DF2
:100E4800410052205F5F2C5F20285F5F2529205FCB
:100E58005F2C5F20285F5F252920206D41004C20F2
:100E68002D5F5F2C5F20285F5F2529202D5F5F2C79
:100E78005F20285F5F252920560052202D5F5F2CB8
:100E88005F20285F5F2529202D5F5F2C5F20285F6A
:100E98005F25292056004C205F5F2C5F2F2D5F5F58
:100EA8002C5F205F5F2C5F2F2D5F5F2C5F206D41D3
:100EB800560052205F5F2C5F2F2D5F5F2C5F205FF5
:100EC8005F2C5F2F2D5F5F2C5F206D4156005057C0
:100ED8004D205F5F205F5F205F5F205F5F20556769
:100EE800313D2D5F5F2C5F2056004368616E67655A
:100EF8002049206176723D5F5F5F2C5F6D41202045
:100F08002020202020004368616E67652049206DFD
:100F180061783D5F5F5F2C5F6D412020202020209D
:100F280020005265737461727420416D706C69663B
:100F38006965722E2E2E2020202020202000537438
:100F48006F702026206469736368617267652E2E4E
:100F58002E20202020202020200056657273696FE3
:100F68006E20496E666F726D6174696F6E2E2E2EDB
:100F7800202020202000496E697469616C697A65B7
:100F880020454550524F4D2E2E2E20202020202027
:100F98002000546F67676C652044656275673A2066
:100FA8005F5F5F2020202020202020202000414457
:100FB8004320303D5F5F5F20313D5F5F5F20323D02
:100FC8005F5F5F20333D5F5F5F0041444320343DF6
:100FD8005F5F5F20353D5F5F5F20363D5F5F5F206D
:100FE800373D5F5F5F00414D3720303D5F5F5F20D9
:100FF800313D5F5F5F20323D5F5F5F20333D5F5F64
:101008005F00414D3720343D5F5F5F20353D5F5FB6
:101018005F20363D5F5F5F20373D5F5F5F00505761
:101028004D2056303D5F5F2056313D5F5F20563280
:101038003D5F5F2056333D5F5F005354502056306C
:101048003D5F5F2056313D5F5F2056323D5F5F2038
:1010580056333D5F5F000F931F932F933F9330915B
:10106800890000270093890010918800130F21E060
:1010780030E100918700002309F4365011230AF467
:10108800122F121708F4122F311708F4132F109388
:1010980088003F912F911F910F9108950F931F93EF
:1010A8002F933F937F938F939F93EF93FF93009199
:1010B8008800000F10E0000F10E0E0EBFDE0E00F0B
:1010C800F11F05911591E02FF12F0995FF91EF91EF
:1010D8009F918F917F913F912F911F910F9108952B
:1010E8000E94C1020E94C60A04E60E94F30906B3E0
:1010F80000FBB6F7089508950E947408002700932E
:1011080089007FEF0E94C10200E87027072F009333
:10111800E5000E94C60A04E60E94F3090E947209CB
:10112800F8943091890000270093890078941091F1
:101138008200130F20918300309184003A95121792
:1011480008F4122F311708F4132F1093820006B3F6
:1011580000FBC6F281E090E0009182000E941E0A26
:101168000E94740808950E9474080027009389005B
:101178007FEF0E94C10200E87027072F0093E50067
:101188000E94C60A04E60E94F3090E947209F894B4
:101198003091890000270093890078941091840089
:1011A800130F2091830035EF121708F4122F31170F
:1011B80008F4132F1093840006B300FBD6F282E0E4
:1011C80090E0009184000E941E0A0E94740808950D
:1011D8000C94290005E000938500C4980895EAE07E
:1011E800F2E11CE6A5E9B0E005910D931A95E1F747
:1011F8000E94C60A12E304E60E94F3091A95D9F779
:101208000895313632352D507573682D50756C6CD4
:101218002020202020202020202020202028632972
:10122800204C617273204D65796572202020202042
:101238002020202020202020666F722041746D65B8
:101248006C2041546D656761203136204020384D4F
:10125800487A2076302E303820204F63742031367B
:1012680020323030382031323A30363A33350E9425
:1012780074080E94C1020FEF0093E5000E94C60A9D
:101288000E94040A0E94740808950E9474080027A6
:10129800009389007FEF0E94C10200E87027072FA2
:1012A8000093E5000E94C60A04E60E94F3090E9422
:1012B8007209F89430918900002700938900789486
:1012C800332321F012F410E001C011E010938700DD
:1012D80006B300FB06F30E9474080895209160008D
:1012E80030916100369527953695279500918400B1
:1012F800201720F007E000938500C4982091620031
:10130800309163003695279536952795009184008E
:10131800201720F008E000938500C498209164000D
:10132800309165003695279536952795009184006C
:10133800201720F009E000938500C49820916600EA
:10134800309167003695279536952795009184004A
:10135800201720F00AE000938500C49820916800C7
:101368003091690036952795369527950AE3021737
:1013780028F00CE000938500C398C49820916A0077
:1013880030916B0036952795369527950DE4021711
:1013980028F00DE000938500C398C49820916C0054
:1013A80030916D00369527953695279504E70217F5
:1013B80028F00EE000938500C398C4982091760029
:1013C8003091770036952795369527950EE50217C3
:1013D80028F00BE000938500C398C49808950F93F4
:1013E8001F932F9328E018EC000000001A95E1F7EE
:1013F8002A95C9F70A95B1F72F911F910F91089572
:101408000F938F939F9381E090E007E3009382000E
:1014180011D082E090E00CED009384000BD09F91F6
:101428008F910F910895E199FECF8EBB9FBBE09AF3
:101438000DB30895F894E199FECF8EBB9FBB0DBB09
:10144800E29AE19A789408950F931F93CF93DF93CC
:101458000F7010E3100F17E00A330AF0010F099319
:10146800DF91CF911F910F9108950F931F932F93A1
:10147800CF93DF93102F12950F701F7020E3020F88
:10148800120F27E00A330AF0020F1A330AF0120F7C
:1014980019930993DF91CF912F911F910F9108957F
:1014A8000F931F932F933F93CF93DF93102F129592
:1014B8000F701F702F7030E3030F130F230F37E0E7
:1014C8000A330AF0030F1A330AF0130F2A330AF00B
:1014D800230F299319930993DF91CF913F912F916E
:1014E8001F910F9108950F931F932F933F934F933D
:1014F8005F93CF93DF93EF93FF934F93CF93DF9354
:101508005FE2000F111F000F111F641711F42CE286
:101518002993259135915395021B130BE0F7020F80
:10152800131F5993000F111F4A9551F7DF91CF915F
:101538004F9110E2461B425032F00881003319F4F3
:1015480019934A95D2F7FF91EF91DF91CF915F916F
:101558005F913F912F911F910F91089500043303DC
:101568008F020C02A301BD0DFD0ACB080807A005D8
:10157800630E820B35095D07E4057002F3018F01E4
:101588003F01FF000F931F937F93AF93BF93A5E98C
:10159800B0E000E80E94530B01E00E94F3097BE1F0
:1015A8000D9191D07A95E1F7A0EBB0E000EC0E94A4
:1015B800530B01E00E94F3097BE10D9184D07A95E9
:1015C800E1F7ABECB0E000E80E945D0B01E00E949F
:1015D800F3097BE10D9183D07A95E1F7A6EEB0E0AF
:1015E80000EC0E945D0B01E00E94F3097BE10D9184
:1015F80076D07A95E1F7BF91AF917F911F910F91C6
:1016080008950F9300E600000000000000000000AD
:101618000A95C9F70F9108950F930FEF04BB0EE1D8
:10162800DEDE00E31CD00AE0DADE00E318D005E0D5
:10163800D6DE00E314D002E0D2DE00E210D002E0F1
:10164800CEDE08E222D002E0CADE0FE01ED002E0C1
:10165800C6DE06E01AD002E0C2DE0F91089505BB8F
:10166800AA9AAB9ACEDFAA98AB98CBDF089505BBB0
:10167800AA9AC7DFAA98AB98C4DF089505BBAB9AAE
:10168800C0DFAA98AB98BDDF08950F930F93007F32
:10169800E6DF0F910295007FE2DF0F9108950F9327
:1016A8000F93007FE4DF0F910295007FE0DF0F9139
:1016B80008950F930F93007FE1DF0F910295007F4C
:1016C800DDDF0F9108950F930F93007F0160CFDF47
:1016D8000F910295007F0160CADF0F9108950F9363
:1016E8000F93007F0160CADF0F910295007F0160B0
:0616F800C5DF0F9108950B
:00000001FF
